:020000040800F2
:10000000B00E00209D010008A5010008A70100080E
:10001000A9010008AB010008AD01000800000000C4
:10002000000000000000000000000000AF01000818
:10003000B101000800000000B3010008B50100088C
:10004000B7010008B7010008B7010008B7010008B0
:10005000B7010008B7010008B7010008B7010008A0
:10006000B7010008B701000885290008B70100089A
:10007000B7010008B7010008B7010008B701000880
:10008000B7010008B7010008B7010008B701000870
:10009000B7010008B7010008B7010008B701000860
:1000A000D9420008F9420008B7010008B70100086A
:1000B000B7010008B7010008B7010008B701000840
:1000C000B7010008B7010008B7010008B701000830
:1000D000B7010008B14700080D480008B701000843
:1000E000B7010008B7010008B7010008B701000810
:1000F000B7010008B7010008B7010008B701000800
:10010000B7010008B7010008B7010008B7010008EF
:10011000A1470008B7010008254300085143000823
:10012000B7010008B7010008B7010008B7010008CF
:10013000B7010008B7010008B7010008B7010008BF
:10014000B7010008B7010008B7010008B7010008AF
:10015000B7010008B7010008B701000839490008D5
:10016000B7010008B7010008B7010008B70100088F
:10017000B7010008B7010008B7010008B70100087F
:10018000B7010008B7010008DFF80CD000F096F9BD
:100190000048004765530008B00E0020064880471D
:1001A00006480047FEE7FEE7FEE7FEE7FEE7FEE75C
:1001B000FEE7FEE7FEE7FEE7D941000889010008F7
:1001C00040EA01039B0703D009E008C9121F08C0D9
:1001D000042AFAD203E011F8013B00F8013B521E59
:1001E000F9D27047D2B201E000F8012B491EFBD2D0
:1001F00070470022F6E710B513460A460446194632
:10020000FFF7F0FF204610BD421C10F8011B00292B
:10021000FBD1801A70472DE9F04D81EA030404F008
:10022000004B21F0004514464FF0000A23F0004136
:1002300050EA050220D054EA01021DD0C5F30A5746
:100240000246C5F31303C1F31300C1F30A5640F489
:10025000801543F48013A7EB0608101BD64608F25E
:10026000FD3873EB050002D308F1010801E0921894
:100270005B41B8F1000F03DA00200146BDE8F08DC4
:1002800000204FF48011064684460EE0171B73EBE6
:10029000050705D3121B63EB050306434CEA010C6B
:1002A00049084FEA300092185B4150EA0107EDD14E
:1002B00052EA030012D082EA040083EA05010843EF
:1002C00005D0101BAB4106D20122002306E000221C
:1002D0004FF0004302E06FF0010253101AEB0600EA
:1002E0004CEB085110EB0A0041EB0B01BDE8F04D5F
:1002F00000F087B80EB5C10F80EAE0700844CA0765
:10030000002140F233438DE80E000A460B4600F010
:1003100087F803B000BD00F0004230F000400AD082
:10032000C10D01F56071C0F3160042EA0151C20827
:1003300040071143704700200146704701F0004319
:1003400030B421F0004150EA010206D00A0DA2F5B6
:100350006072C1F31301002A02DC30BC0020704738
:10036000440F44EAC104C100E01830BC00EBC250A5
:1003700000F010B8202A04DB203A21FA02F0002114
:10038000704721FA02F3D040C2F1200291400843A5
:10039000194670470029A8BF7047401C490008BF94
:1003A00020F00100704710B4B0FA80FC00FA0CF0A5
:1003B00050EA010404BF10BC704749B1CCF12004DD
:1003C00021FA04F411FA0CF118BF0121214308436A
:1003D000A3EB0C01CB1D4FEA00614FEA102042BF96
:1003E000002010BC704700EBC35010440029A4BF8C
:1003F00010BC7047401C490008BF20F0010010BC31
:10040000704710B5141E73F1000408DA401C41F166
:10041000000192185B411A4301D120F0010010BD88
:100420002DE9F04D92469B4611B1B1FA81F202E0FE
:10043000B0FA80F22032904600F052F804460F469F
:1004400040EA0A0041EA0B0153465A46084313D0DA
:10045000114653EA010019D0C8F140025046FFF797
:1004600089FF05460E4650465946424600F038F888
:10047000084305D0012004E020463946BDE8F08D50
:100480000020054346EAE0762C4337430A9863058B
:10049000E40AA0EB08000022FD0A44EA47540A30AF
:1004A00002D500200146E9E7010510196941DDE99F
:1004B000084500196941BDE8F04DA2E7064C074D1B
:1004C00006E0E06840F0010394E807009847103424
:1004D000AC42F6D3FFF75CFED8570008F857000887
:1004E000202A04DB203A00FA02F1002070479140F4
:1004F000C2F1200320FA03F319439040704770B50E
:100500008D1810F8014B14F0030201D110F8012BE3
:10051000231106D110F8013B03E010F8016B01F83C
:10052000016B521EF9D1ABB110F8012B04F00C0491
:100530008A1A0C2C03D0A2EB84129B1C08E010F842
:10054000014BA2EB0422F8E712F8014B01F8014B32
:100550005B1EF9D5A942D4D3002070BDCA43026006
:10056000704721B1826842F00102826003E0826834
:1005700022F00102826070470021084A1168084A8F
:100580001140D0E900231A4383681A43C3681A4311
:100590001143044AC2F804137047000004230140C9
:1005A000E030FCFF0020014000B58DB0012108467D
:1005B00003F09AFA0121080203F0C6FA40200190E4
:1005C00003208DF8080000208DF80B0001A91748C2
:1005D00002F015FB0020039004900690059003A8FC
:1005E000FFF7CAFF0121080203F0BEFA00214FF411
:1005F000807003F0B9FA00208DF8200007908DF884
:10060000210009900B9001208DF8300007A90848BF
:1006100000F01EF8062301221946054800F042F8B2
:1006200001210348FFF79DFF0DB000BD000002400F
:10063000002001400146C86C80B27047024600208D
:1006400013680B400BB1012000E000207047000050
:1006500030B50246002000235068104C20400D7930
:100660000C6844EA05242043506090680C4C2040FC
:10067000D1E903542C438D682C434D7944EA450459
:1006800020439060D06A20F470000C7D641EE4B2B8
:10069000234340EA0350D06230BD0000FFFEFFFC60
:1006A000FDF7FFC0F0B504460D4600200021092DDE
:1006B00011DDE068A5F10A0606EB4607072606FAF3
:1006C00007F18843A5F10A0606EB460603FA06F190
:1006D0000843E0600CE0206905EB4507072606FAB1
:1006E00007F1884305EB450603FA06F1084320614C
:1006F000072A0FDA606B561E06EB86071F2606FADE
:1007000007F18843561E06EB860605FA06F10843F4
:10071000606322E00D2A0FDA206BD61F06EB8607F6
:100720001F2606FA07F18843D61F06EB860605FA50
:1007300006F10843206310E0E06AA2F10D0606EB23
:1007400086071F2606FA07F18843A2F10D0606EB7D
:10075000860605FA06F10843E062F0BD816841F0C3
:10076000804181607047000070B50023224A1278F2
:10077000082A03DA0022214C22703BE0002034E0FA
:100780001F4A125C552A2ED11D4CC21DA25CBB2AE9
:1007900029D12546841C2D5D194EC41C345D254489
:1007A000041D345D2544441D345D2A19D41702EB21
:1007B00014642412A2EB0424E3B23446821DA25C2A
:1007C0009A420DD1002105E00A180D4CA25C62543A
:1007D0004A1CD1B20829F7DB0122084C227002E042
:1007E0000022064C2270421CD0B2034A1278D21F5B
:1007F0008242C5DA70BD0000F0040020060500202A
:100800002009002010B500F009F8012003F0A6FC33
:1008100000200149086010BDBC0243421CB5012103
:10082000422003F061F94020009001208DF804007F
:1008300000208DF8060003208DF8050069460A485F
:1008400002F0DDF94FF40040009001208DF8040023
:1008500000208DF8060003208DF805006946024847
:1008600002F0CDF91CBD00000004024010B503F0F9
:10087000CFFA012008490860022004F03BFD074838
:10088000D0F81C02C4B2002003490860022004F022
:1008900031FD204610BD0000988240420080404259
:1008A00070B5002403F0B4FA012010490860002557
:1008B00017E06006040E01200C49091F08600220A1
:1008C00004F018FD0A48D0F81C0208B1601CC4B23C
:1008D00000200649091F0860022004F00BFD681C77
:1008E000C5B2082DE5DB204670BD00009C82404269
:1008F0000080404210B5044603F09AFA1CB1012072
:100900000A49086002E00020084908600120074900
:10091000091F0860022004F0EDFC00200449C1F822
:100920009802022004F0E6FC10BD00009C824042C8
:100930000080404270B5044603F07AFA00251BE0BF
:1009400004F080061EB101200E49086002E000207C
:100950000C4908606006040E01200A49091F08605E
:10096000022004F0C7FC00200749C1F898020220C9
:1009700004F0C0FC681CC5B2082DE1DBFFF776FF70
:1009800070BD00009C8240420080404210B503F0E0
:100990004FFA0120094908600949C1F8980204206A
:1009A00004F0A8FC002005490860042004F0A2FC23
:1009B00000200349C1F8980210BD00009C8240420B
:1009C0000080404210B503F033FA00200749086068
:1009D00001200749C1F89802042004F08BFC012093
:1009E00002490860042004F085FC10BD9C8240424E
:1009F0000080404210B503F047FF10BD10B504461B
:100A00000B48844209D10121480603F08DF80021EA
:100A10004FF0007003F088F808E00121880603F029
:100A200083F800214FF0806003F07EF810BD0000D5
:100A30000064004010B50021837A012202FA03F11C
:100A40003D4A126842F001023B4B1A603A4A1C329E
:100A500012688A43384B1C331A60027BCAB9364A83
:100A60000C3212688A43344B0C331A604288C388B4
:100A700042EA0343304A4032847A42F834300288F2
:100A8000838842EA03432C4A4032847A02EBC40250
:100A90005360027B012A19D1274A0C3212680A439B
:100AA000254B0C331A604288038842EA0343224AEA
:100AB0004032847A42F83430C288838842EA034361
:100AC0001D4A4032847A02EBC4025360C27A3AB9BA
:100AD000194A121D12688A43174B1B1D1A6006E043
:100AE000154A121D12680A43134B1B1D1A60028916
:100AF00032B9114A143212688A430F4B14331A6008
:100B00000289012A06D10C4A143212680A430A4BA0
:100B100014331A60427B012A06D1074A1C3212683C
:100B20000A43054B1C331A60034A126822F0010283
:100B3000014B1A6010BD0000006600401AB1436905
:100B40000B43436102E043698B434361704730B517
:100B5000024600200023146824F002041460146884
:100B600044F00104146000E05B1C546804F00104CC
:100B70001CB94FF6FF74A342F6D1546804F0010487
:100B80000CB900206CE08C79012C04D1146844F07D
:100B90008004146003E0146824F080041460CC79AD
:100BA000012C04D1146844F04004146003E014687C
:100BB00024F0400414600C7A012C04D1146844F031
:100BC0002004146003E0146824F0200414604C7ABC
:100BD000012C04D1146844F01004146003E014687C
:100BE00024F0100414608C7A012C04D1146844F0B1
:100BF0000804146003E0146824F008041460CC7A3C
:100C0000012C04D1146844F00404146003E0146857
:100C100024F0040414608C78A407CD7844EA0564B9
:100C20000D7944EA05444D7944EA05540D886D1E5A
:100C30002C43D461146824F001041460002300E004
:100C40005B1C546804F001041CB14FF6FF74A3420E
:100C5000F6D1546804F001040CB1002000E001203A
:100C600030BD0246002019B9D36803F0030006E046
:100C7000012903D1136903F0030000E0002070474D
:100C800010B500F5D87303EB01131B6803F00403E0
:100C90001372137A53B900F5D87303EB01131B6871
:100CA00040F2FF7404EA5353136009E000F5D8736F
:100CB00003EB01131B686FF0604404EAD303536035
:100CC00000F5D87303EB01131B6803F002035372A2
:100CD00000F5D87303EB01135B6803F00F03937205
:100CE00000F5D87303EB01135B681B0AD37400F59E
:100CF000D87303EB01139B68D37200F5D87303EB31
:100D000001139B681C0A147300F5D87303EB0113DD
:100D10009B681C0C547300F5D87303EB01139B689C
:100D20001B0E937300F5D87303EB0113DB68D373C9
:100D300000F5D87303EB0113DB681C0A147400F58B
:100D4000D87303EB0113DB681C0C547400F5D873E3
:100D500003EB0113DB681B0E937421B9C36843F0E6
:100D60002003C36003E0036943F02003036110BD67
:100D700010B502460020936803F08063B3F1806FE2
:100D800000D110E0936803F00063B3F1006F01D16C
:100D9000012008E0936803F08053B3F1805F01D134
:100DA000022000E00420042874D002F5C07303EB95
:100DB00000131B6803F0010402F5C07303EB00137A
:100DC0001C600B7A7BB94B7A0C8843EA445302F5DA
:100DD000C07404EB00142468234302F5C07404EBD0
:100DE0000014236010E00B7A4C6843EAC4034C7A89
:100DF000234302F5C07404EB00142468234302F576
:100E0000C07404EB001423608B7A03F00F038B7221
:100E100002F5C07303EB00135B6823F00F0402F5C7
:100E2000C07303EB00135C6002F5C07303EB0013A7
:100E30005B688C7A234302F5C07404EB0014636092
:100E40008B7B1C064B7B44EA03440B7B44EA032365
:100E5000CC7A234302F5C07404EB0014A3608B7CAE
:100E60001C064B7C44EA03440B7C44EA0323CC7B02
:100E7000234302F5C07404EB0014E36002F5C07371
:100E800003EB00131B6843F0010402F5C07303EB8E
:100E900000131C6010BD000010B50246002321B1F4
:100EA000012907D002290FD109E090681D4C00EA02
:100EB00004030BE090681C4C00EA040306E0906811
:100EC0001A4C00EA040301E0002300BF00BF184CE5
:100ED000181BA34216D007DC83B16FF08060184462
:100EE00070B1022818D111E0B0F5007F10D0114C7C
:100EF000204448B1B0F5003F0ED10BE002230DE0D5
:100F000000230BE0002309E0002307E0012305E0B4
:100F1000012303E0012301E0002300BF00BFD8B29A
:100F200010BD0000030000040003000800000310CF
:100F3000000100080001FFF72DE9FF4705460E46B6
:100F40004FF0000A06B10DB94FF0010A944800783D
:100F500000F00F00032801DD4FF0010A90480078EF
:100F6000C0F30019BAF1000F19D000208DF80A0063
:100F70008DF80B0001208DF80C000020ADF800006A
:100F8000ADF80200ADF80400ADF80600ADF80800B9
:100F900001208DF80D006846FFF74CFDFEE00020B3
:100FA000ADF8080001208DF80D004FF00008002476
:100FB000F2E07B48007800F00F0030B101283BD010
:100FC00002287BD0032874D19CE000208DF80B0010
:100FD0008DF80C0035F824004B460022114600F035
:100FE000E1F8ADF8020005EB840148884B46002289
:100FF000114600F0D7F8ADF80600601CC0B20446F8
:10100000B04213DA35F824004B460022114600F0B6
:10101000C9F8ADF8000005EB840148884B46002272
:10102000114600F0BFF8ADF8040004E00020ADF870
:101030000600ADF804009CE001208DF80B000020B4
:101040008DF80C0035F824004B460022114600F0C4
:10105000A9F8ADF80200601CC0B20446B04207DA3D
:1010600035F824004B460022114600F09BF800E0C2
:101070000020ADF80600601CC0B20446B04207DA9A
:1010800035F824004B460022114600F08BF800E0B2
:101090000020ADF80000601CC0B20446B04209DA7E
:1010A00035F824004B460022114600F07BF802E0A0
:1010B00004E051E00020ADF804005AE000208DF873
:1010C0000B0001208DF80C0035F824004B4600225F
:1010D000114600F081F80746B8B2ADF80200380CAE
:1010E000ADF8000005EB840148884B46002211460C
:1010F00000F072F80746B8B2ADF80600380CADF84B
:10110000040036E001208DF80B008DF80C0035F856
:1011100024004B460022114600F05EF80746B8B2A4
:10112000ADF80200380CADF80000601CC0B20446F7
:10113000B04208DA05EB840148884B46002211468C
:1011400000F04AF800E000200746B8B2ADF806000B
:10115000380CADF804000CE00020ADF80200ADF84A
:101160000000ADF80600ADF8040034464FF0010A67
:1011700000BF00BF8DF80A806846FFF75BFCB442F1
:1011800002DA601CC4B200E007E008F10100C0B25E
:1011900080460D2800DB00E00BE700BFBDE8FF87BD
:1011A0008803002010B50446C4F309040AB11020D6
:1011B00000E0002002460BB1082000E000200346BA
:1011C00013B1C1F3C13000E00020014642EA4410EF
:1011D0001843084380B210BD10B50446C4F3090497
:1011E0000AB1022000E0002002460BB1042000E01A
:1011F0000020034613B18803C00A00E00020014626
:1012000042EA44301843084310BD000010B50021E5
:101210000148FFF726FD10BD0064004070B504468C
:10122000002554B100210648FFF71BFD054625B1F6
:10123000224600210248FFF723FD284670BD00002A
:10124000006400402DE9F04706460C4617469846D4
:10125000DDF820904FF0000A15480760C0F80480C0
:1012600000201349087248720846847222463146AB
:101270000B30FEF7A5FF0E490E48FFF779FD054636
:10128000042D09D04FF0010A29460A48FFF704FE51
:10129000012801D14FF0020ABAF1010F04DBB9F1C4
:1012A000000F01D089F800505046BDE8F0870000DB
:1012B000C4060020006400400448006800F0E050CC
:1012C00008B1012070470020FCE7000008640040DE
:1012D00010B501E000F006F8FFF798FF0028F9D1FB
:1012E00010BD000010B52448FFF798FF2248C07CCD
:1012F00020B101280AD0022818D10FE01E48827AB6
:1013000000F10B011D4801F0EEFB24E01A48827A3F
:1013100000F10B011A4801F0E6FB1CE01648827A46
:1013200000F10B01174801F0DEFB14E01248C07C0D
:1013300003280FDB1048C07C06280BDC0E48C07C5D
:10134000C01E114901EBC0000B490B310A68026055
:101350004968416000BF00BF0748C07C062809DC1F
:101360000548C07C094951F820000949096808432B
:101370000749086010BD000038080020EC06002076
:10138000FC0600201C0700204C080020C85600085E
:101390008C03002000B5034A5178107801F05AFF01
:1013A00000BD00004C080020F8B5FFF785FF0028BD
:1013B0005FD00026002559E02E4890F9000030B19A
:1013C00001280ED002281ED0032840D12DE000F0C5
:1013D0005DF80746002F03DB0126F8B200F07AF82B
:1013E00039E008222449254801F068FBC4B24CB119
:1013F0000126234800234FF42072214600901E4806
:10140000FFF720FF27E008221B491E4801F056FB8A
:10141000C4B24CB101261A4800234FF42872214669
:1014200000901548FFF70EFF15E0082212491648F4
:1014300001F044FBC4B24CB10126114800234FF423
:101440007072214600900C48FFF7FCFE03E0FF207D
:101450000849087000BF00BF06480078401C40B231
:101460000449087006B103E0681CC5B2042DA3DD71
:1014700000BFF8BDC0030020900300200C0700202F
:10148000C10300202C070020EC0600204FF0FF30A5
:10149000002109E001EB8102054B13F822200AB17B
:1014A00048B203E04A1CD1B20729F3DB00BF704702
:1014B0006C080020002007E0002100EB8002044BB4
:1014C00003F82210411CC8B20728F5DB7047000062
:1014D0006C080020F8B50446002004EB84050E4E8D
:1014E00006EB850500902B6904EB840506EB85056A
:1014F000EA6804EB840516F8251004EB840506EB76
:101500008505681CFFF79EFE002004EB840132462F
:1015100002F82100F8BD00006C0800202DE9F04120
:1015200004460F4615461E46DDF81880072C1ADAC9
:1015300004EB84000D4901F8205004EB84010B4AB0
:1015400002EB8101481C2A463946FEF739FE04EBBE
:101550008400064901EB8000C66004EB840001EBC7
:101560008000C0F81080BDE8F08100006C08002009
:1015700010B50D4A32210D4800F02AF80C4A3221EC
:101580000C4800F025F80C4A32210C4800F020F8F5
:101590000B4A32210B4800F01BF80B4A32210B4852
:1015A00000F016F810BD00003C070020EC060020FB
:1015B0006E070020FC060020A00700200C0700207A
:1015C000D20700201C070020040800202C07002060
:1015D00070B504460E4615462660E560002120469B
:1015E00001F0BBFA70BD000038B5FFF771FE68E08E
:1015F000FFF76EFE002462E0344850F824003449BE
:1016000009680840002858D0072C4DD2DFE804F0C4
:10161000040C18242739460000BF69462D4801F004
:10162000AEFA0028F9D13FE003E09DF8000000F099
:101630007BFA6946284801F0A2FA0028F5D133E088
:1016400003E09DF8000000F0A3FB6946234801F089
:1016500096FA0028F5D127E0FFF79CFE24E0204809
:1016600003F096F81F49088005E01E480088A0F5A1
:1016700061601C4908801B480088B0F5616FF4DA8E
:1016800012E017480838007C022806D114480930B7
:1016900003F076F800B21449088005E010480838D5
:1016A000007E012800D100BF00BF104850F8240080
:1016B00007490968084006490860601CC4B2062C46
:1016C0009ADD03480068002892D138BDC85600084A
:1016D0008C030020EC060020FC0600201C070020E4
:1016E000540800209C0300209A030020485700085B
:1016F00010B5002006490860064908700721064811
:10170000FFF71AFCFFF734FFFFF7D4FE10BD00000F
:101710008C030020880300209E03002010B5EB48B6
:101720000078E0B1EA48006803F010FEB8B9E94873
:101730000078FD2807D1E8480078401CC1B2E54890
:1017400002F028FC08E0E3480078552802D101F0B7
:10175000FFFF01E0FFF708F80020DC490870DF48D0
:10176000007801287ED1DB484078AA287BD1D9486F
:101770008078122878D00CDC122876D2DFE800F0CE
:101780007522295896B2CFE4E5FE757575757575A5
:10179000FDFC61286AD00CDC402868D004DC2028DD
:1017A00066D0302861D15FE150287BD05128F9D133
:1017B00065E1622877D0632876D0802875D0A0288C
:1017C000F0D175E10021084602F0AEFB02F0CAFA42
:1017D00073E102F009FB0020C14908700120C149F2
:1017E00008700020C0490870C0490870C0490870DE
:1017F000C0490870C0490870B6484079BF490880A0
:10180000084600884FF6FF7101EA0020BB490880B6
:10181000B048007909880843B8490880AD48C078C5
:10182000B749086008460168006801F030F844E1F3
:1018300002F0DAFA0020AA490870AA490870AA49F9
:101840000870AA490870AA4908700120A9490870BF
:101850000020A94908709F484079A8490880084697
:10186000008806E031E129E1EEE025E10CE100E14C
:10187000EFE04FF6FF7101EA0020A049088095488B
:101880000079098808439D4908809248C0789C499E
:10189000086008460068414299480068404200F0EC
:1018A000F6FF0AE1E6E0F4E0F8E0FCE000208C4915
:1018B00008708C49087001208B49087000208B4902
:1018C00008708B4908708B4908708B4908708148F3
:1018D000C0788B490860084601680068404200F003
:1018E000D6FFEAE000207E4908707E4908707E49F4
:1018F000087001207D49087000207D4908707D49ED
:1019000008707D4908707348C0787D4908600846B2
:10191000006841427A48006800F0B9FFCDE000203D
:101920006F4908706F4908706F4908706F490870F7
:101930006F4908706F49087001206F490870654849
:10194000C0786F490860B8E0B7E002F057FA02F0DB
:101950004BFA0020624908706249087062490870B9
:1019600062490870012062490870002061490870CE
:1019700061490870574802E05BE04FE01BE04079A6
:1019800060490880084600884FF6FF7101EA002090
:101990005C4908804F480079098808435949088004
:1019A0004C48C078564908600846016800684042C3
:1019B00002F0BAFA81E002F021FA02F015FA0020F2
:1019C00047490870474908704749087047490870F7
:1019D00001204749087000204649087046490870B0
:1019E0003C48407947490880084600884FF6FF7117
:1019F00001EA0020434908803648007909880843F5
:101A0000404908803348C0783D490860084600686E
:101A100041423B48006802F087FA4EE02D48C0780A
:101A2000394908702B48007948702A4840798870F5
:101A300043E02848C0783449C870264800790871C6
:101A400024484079487138E006212F4801F028FCED
:101A500033E02048C178012002F05AFB1D4801798B
:101A6000022002F055FB28E01A49C87802F03EFB3C
:101A700023E022E00421254801F012FC1DE00421AE
:101A8000234801F00DFC18E00421224801F008FC75
:101A900013E00421204801F003FC0EE004211F485C
:101AA00001F0FEFB09E00B48C0781D49087004E016
:101AB00001201C49087000E000BF03E00821054830
:101AC00002F068FA00200549087010BDF1040020FA
:101AD000F804002020090020F00400200605002062
:101AE0006A0300205F0300205C0300205D030020E8
:101AF0005E030020600300206103002078030020C3
:101B0000740300207A03002007050020B804002099
:101B1000C0040020C4030020C8030020CC03002020
:101B2000F40400204201002010B504460F4800785C
:101B300070B903F005FC0A300D49086000200D491A
:101B400008700D48097844540120084908700BE0DA
:101B500008480078C82807DA06480078401CC0B258
:101B60000449087004490C5410BD0000F104002021
:101B7000F8040020F00400202009002010B57A4865
:101B80000078002879D07948006803F0DFFB00284E
:101B900073D177484078032808D1754880780128A8
:101BA00003D17348007973490870D9E070484078D0
:101BB0000C280CD16E4880780128F6D16C48C0788A
:101BC0000128F2D16A4800796A490870C8E068487B
:101BD00040780E2808D166488078012804D16448EE
:101BE000007964490870BBE06148407810280CD146
:101BF0005F488078102808D15D48C0780128D4D18A
:101C00005B4800795B490870AAE0594840780D2884
:101C100058D157488078032854D15548C0780128B6
:101C20001BD153480079012806D0022808D0032888
:101C30000AD0042810D10BE009204E4908700BE0AF
:101C40000A204C49087007E00B204A49087003E05D
:101C50000C204849087000BF82E04548C07802283F
:101C60007ED143480079012808D1414840790128B4
:101C700004D111203F49087072E074E03C480079BB
:101C8000022807D13A484079022803D12220394955
:101C9000087065E036480079012807D1344840795A
:101CA000022803D112203349087059E030480079E6
:101CB000022855D12E484079012851D121202D49A3
:101CC00008704DE02A484078072808D128488078D5
:101CD000012804D12648C0782749087040E02448EC
:101CE000007855280CD122484078022808D13222A9
:101CF0001F492248FEF764FA0120214908702FE0AD
:101D00001B484078062808D119488078012827D137
:101D10001748C0781749087022E015484078012814
:101D20001ED113488078A8281AD1002413E001207E
:101D3000144908604FF4FA7003F0B6FA0020124913
:101D4000C1F894024FF4FA7003F0AEFA00200F4984
:101D50000870601CC4B2032CE9DBA8200B49087092
:101D600000200149087010BDF3040020FC0400208D
:101D7000E80900206A0300204501002052060020E7
:101D8000F504002094824342008043424201002037
:101D900010B504460F48007870B903F0D1FA0A3044
:101DA0000D49086000200D4908700D480978445419
:101DB0000120084908700BE008480078C82807DAB5
:101DC00006480078401CC0B20449087004490C540D
:101DD00010BD0000F3040020FC040020F2040020E9
:101DE000E80900207FB505460C460121202001F0BE
:101DF0008BFE0295ADF804400020ADF80600ADF86A
:101E00000C008DF80E0001A90D4802F0DBFA372016
:101E10008DF8000000208DF8010004208DF80200EC
:101E200001208DF80300684601F04CFC01221146A8
:101E3000034802F0BDFA0121014802F09CFA7FBD7F
:101E40000014004010B5FFF7CFFBFFF7ADFA10BD4F
:101E500070B504460D4601F0C7FF00201149087017
:101E6000114908701149087011490870114908702A
:101E700001201149087000201049087010480580A1
:101E800010480460006841420E480068404200F07B
:101E9000FEFC02E0642003F007FA02480078032801
:101EA000F8D170BD6A0300205F0300205C030020AE
:101EB0005D0300205E03002060030020610300201A
:101EC000780300207403002070B504460D4601F02D
:101ED0008BFF00200E49087001200E490870002079
:101EE0000D4908700D4908700D4908700D490870BA
:101EF0000D4908700D4805800D48046001680068B0
:101F000000F0C5FC00BF024800780328FBD170BD7B
:101F10006A0300205F0300205C0300205D030020B3
:101F20005E0300206003002061030020780300208E
:101F30007403002010B5044601F056FF00200E493E
:101F400008700E49087001200D49087000200D49E5
:101F500008700D4908700D4908700D4908700D484A
:101F6000046001680068404201F0DEFF00BF0248E3
:101F700000780228FBD110BD6A0300205F03002017
:101F80005C0300205D0300205E030020600300204E
:101F9000610300207403002010B5044601F024FF03
:101FA00000200F4908700F4908700F490870012080
:101FB0000E49087000200E4908700E4908700E493D
:101FC00008700E480460006841420C48006801F047
:101FD000ABFF00BF024800780228FBD110BD000013
:101FE0006A0300205F0300205C0300205D030020E3
:101FF0005E030020600300206103002074030020C2
:1020000010B5FE480078A6287DD0F6287CD108219E
:10201000FB4801F0BFFFC82003F046F90821F8484B
:1020200001F0B8FFC82003F03FF9F648007800F04F
:10203000B3FBF5480188F3480078FFF745FF4FF4FC
:10204000FA7003F031F90020F0490860F048007898
:10205000FFF770FF4FF4FA7003F026F900210846ED
:1020600000F015FC0120EB49C1F8A8024FF4FA700A
:1020700003F01AF94FF448711E2000F045FB4FF4AD
:10208000FA7003F011F90821E34801F083FF4FF4DF
:10209000FA7003F009F90821E04801F07BFF4FF4E2
:1020A000FA7003F001F90021084600F0F0FB43F656
:1020B000982003F0F9F80821D74801F06BFF4FF49E
:1020C000FA7003F0F1F80821D54801F063FF40F2FF
:1020D000DC5003F0E9F8CB48007800F05DFBCA481B
:1020E0000188C8480078FFF7EFFE4FF4FA7003F05C
:1020F000DBF8CCA001F080FC4FF4FA7003F0D4F8C8
:102100000020C44901E0C5E1E0E2C1F8A802C048EE
:102110000078FFF70FFF4FF4FA7003F0C5F80021C5
:10212000084600F0B4FB0120BA49C1F8A8024FF4F8
:10213000FA7003F0B9F80621BE4801F0B1F84FF487
:102140007A7003F0B1F85A20FFF7F4FE4FF4FA70FA
:1021500003F0AAF80021084600F099FB4FF4FA704A
:1021600003F0A2F8A748007800F016FBA648018803
:10217000A4480078FFF7A8FE4FF4FA7003F094F833
:1021800000F060FEACA000F073FEC82003F08CF8F5
:10219000A9A000F06DFE4FF4167003F085F8012140
:1021A000202003F00FF89748007800F0F5FA9648E1
:1021B000018894480078FFF787FE4FF4FA7003F027
:1021C00073F8C82003F070F800209249C1F8AC02FF
:1021D0008F480078FFF7E0FE4FF4FA7003F064F8E0
:1021E0000021084600F053FB01208849091D0860C2
:1021F0004FF4FA7003F058F88248007800F0CCFAF7
:10220000814801887F480078FFF75EFE4FF4FA703E
:1022100003F04AF800207F49C1F8A8027C48007802
:10222000FFF788FE4FF4FA7003F03EF800210846ED
:1022300000F02DFB4FF4FA7003F036F801207549D9
:10224000C1F8A802C82003F02FF8032001F08CF990
:10225000C82003F029F85020FFF79EFE4FF4FA70D3
:1022600003F022F80021084600F011FB4FF4FA7049
:1022700003F01AF840F2DC51142000F045FA4FF454
:10228000FA7003F011F80021084600F000FB41F25B
:10229000883003F009F86AA002F0BEFF59480078C0
:1022A00000F07AFA4FF4FA615020FFF70DFE4FF478
:1022B000FA7002F0F9FF00205649C1F8A80254480C
:1022C0000078FFF737FE4FF4FA7002F0EDFF0021BF
:1022D000084600F0DCFA01204C4908604FF4FA701F
:1022E00002F0E2FF4748007800F056FA46480188BD
:1022F00044480078FFF7E8FD4FF4FA7002F0D4FF8D
:1023000000204449C1F8A80241480078FFF712FEB6
:102310004FF4FA7002F0C8FF0021084600F0B7FA47
:1023200001203C49C1F8A8024FF4FA7002F0BCFF4A
:102330004FF47A71142000F0E7F900F0D7FA4FF467
:10234000FA7002F0B1FF2F48007800F025FA2E480D
:1023500001882C480078FFF7B7FDC82002F0A4FFE1
:102360002848007800F018FA2748018825480078A6
:10237000FFF7AAFD4FF4FA7002F096FF00202549FE
:10238000C1F8A80222480078FFF7D4FD4FF4FA7094
:1023900002F08AFF0021084600F079FA01201D4969
:1023A000C1F8A8024FF4FA7002F07EFF4FF47A7180
:1023B00014480078FFF74CFD4FF4FA7002F074FFF8
:1023C0000121412000F094FC642002F06DFF0821FF
:1023D000224801F0DFFD4FF4967002F065FF0821FE
:1023E0001E4801F0D7FD4FF4FA7002F05DFF08219E
:1023F0001B4801F0CFFDC82034E00000420100205E
:102400003C0000203C0100203E010020A882434205
:102410003D01002000804342540000205C00002069
:1024200064000020C7B0B7BDCEDEB7A8CDA8D0D01D
:10243000000000000C000020413131343531000033
:10244000BCB4BDABCDA8D0D0B9FDB0DFC2EDCFDFFD
:10245000A3ACC7EBD7A2D2E20000000044000020EA
:102460000401002002F020FF0821994801F092FDAC
:10247000C82002F019FF97A002F0CEFE4FF4FA70C8
:1024800002F012FF00210846FFF71EFD00209449CC
:1024900008701BE10021412000F02AFC082191482E
:1024A00001F078FDC82002F0FFFE08218D4801F000
:1024B00071FD42F2107002F0F7FE8B48007800F0D8
:1024C0006BF98A48018888480078FFF7FDFC4FF4D3
:1024D000FA7002F0E9FE002085490860854800781E
:1024E000FFF75AFD4FF4FA7002F0DEFE00210846B5
:1024F00000F0CDF901208049C1F8AC024FF4FA7028
:1025000002F0D2FE02F0DCFD7C4800887C490880A5
:1025100008460188412001F093FEC82002F0C4FE65
:102520007748008800F0DCFF75480188412001F001
:1025300087FE4FF4FA7002F0B7FE00206E49C1F832
:10254000A8026C480078FFF7F5FC4FF4FA7002F02F
:10255000ABFE0021084600F09AF901206649C1F857
:10256000A8024FF4FA7002F09FFE5F48007800F076
:1025700013F95E4801885C480078FFF7A5FC5A48CB
:10258000007800F009F95948018857480078FFF7AA
:102590009BFC4FF4FA7002F087FE00205649C1F808
:1025A000AC0254480078FFF7F7FC4FF4FA7002F0E1
:1025B0007BFE0021084600F06AF901204E49C1F86F
:1025C000AC024FF4FA7002F06FFE02F079FD4B4856
:1025D00000884B49088008460188422001F030FEFF
:1025E000C82002F061FE4648008800F079FF4448A8
:1025F0000188422001F024FE4FF4FA7002F054FEEC
:102600002820FFF7C9FC4FF4FA7002F04DFE0021BC
:10261000084600F03CF93448007800F0BDF8334833
:10262000018831480078FFF74FFC2F48007800F010
:10263000B3F82E4801882C480078FFF745FC4FF48A
:10264000FA7002F031FE5020FFF7A6FC4FF4FA704A
:1026500002F02AFE2820FFF79FFC4FF47A712248EF
:102660000078FFF7F5FB0121412000F041FB6420D9
:1026700002F01AFE0821234801F08CFC4FF49670FA
:1026800002F012FE08211F4801F084FC4FF4FA709A
:1026900002F00AFE08210E4801F07CFCC82002F07E
:1026A00003FE08210A4801F075FCC82002F0FCFD79
:1026B00008A002F0B1FD4FF4FA7002F0F5FD002120
:1026C0000846FFF701FC00200549087000BF10BD57
:1026D00004010020BDE1CAF8C8CECEF10000000020
:1026E000420100203C0000203C0100203E0100206F
:1026F000AC8243423D01002000804342D0010020D3
:10270000400100204400002070B505460C46002022
:102710001949087019490870194908701949087051
:102720001949087019490870012019490870194899
:1027300005600168006800F0AAF840F21630844293
:1027400003DC204602F0B0FD08E040F2163002F053
:10275000ABFDA4F2163188B202F0A6FD01F002FB37
:102760000021084601F0E0FB0120034908706420C5
:1027700002F09AFD70BD00006A0300205F03002094
:102780005C0300205D0300205E0300206003002046
:10279000610300207403002010B5044601F024FBFF
:1027A00000200D4908700D4908700D4908700D4949
:1027B00008700D4908700D49087001200C49087017
:1027C0000C4804600168006800F061F800BF02482E
:1027D00000780128FBD110BD6A0300205F030020B0
:1027E0005C0300205D0300205E03002060030020E6
:1027F00061030020740300201CB501214FF4C07058
:1028000001F072F9F020009000208DF80400012002
:102810008DF807006946144800F0F1F94FF4704054
:10282000009001208DF8040000208DF806000120A2
:102830008DF8070003208DF8050069460B4800F06D
:10284000DEF92020009001208DF8040000208DF892
:10285000060001208DF8070003208DF80500694669
:10286000024800F0CCF91CBD00200240001C0240D0
:1028700070B505460C460026284601F023FA0646A8
:1028800026EA0401284602F073FC002070BD70B5F2
:1028900005460C46002D06DB642D00DD6425052D64
:1028A0000BDA052509E015F1640F01DA6FF0630515
:1028B00015F1050F01DD6FF00405002C06DB642C1B
:1028C00000DD6424052C0BDA052409E014F1640F03
:1028D00001DA6FF0630414F1050F01DD6FF00404F9
:1028E0002146284601F020FB70BD000070B5002590
:1028F000002431E002F024FD00F57A7513E017485A
:10290000007801280FD1002014490870144840783D
:102910000C2808D112488078012804D10E2111A07A
:1029200001F0F4FA70BD284602F010FD0028E6D14F
:10293000601CC4B2032C04DB16210DA001F0E6FAE2
:10294000F0E764212820FFF783FA642002F0ACFC52
:102950006E212820FFF7B8FACCE70000F30400202E
:10296000E8090020455443737563636565640A0094
:10297000455443636F6E74726F6C206661696C6559
:10298000640A000010B5102000F03CF8012825D1A1
:102990001021134800F09EF9E8B90021114801F018
:1029A000EAFC114890ED000AB8EE400A0F4880EDAD
:1029B000000AD0ED000A9FED0E1AB3EE040A10EEE5
:1029C000810A80ED000A90ED000ABCEEC00A10EE0C
:1029D000100A08490880102000F00EF810BD000011
:1029E0000004024000100040CC010020C80100207B
:1029F000F628DC3FD0010020014908607047000044
:102A0000143C014001460020034A12680A400AB102
:102A1000012000E000207047143C014000212349C0
:102A20008279002A3AD00A46126803689A430B4614
:102A30001A600A1D126803689A430B1D1A60027916
:102A400011440A6803681A430A60184A0832126877
:102A500003689A43154B08331A601A1D12680368FD
:102A60009A43124B0C331A604279102A0ED11A1F66
:102A7000126803681A430D4B08331A601A1D126856
:102A800003681A43094B0C331A600DE00749427979
:102A900011440A6803681A430A6005E00279114488
:102AA0000A6803689A430A6070470000003C0140CE
:102AB00010B500F075FEFDF777FD10BDF0B50746C7
:102AC0000C461646002564B106E06119384600F050
:102AD00056F800B904E06D1C301EA6F10106F4D1D1
:102AE00000BF2846F0BDF0B507460D461646002447
:102AF00006E0295D384600F06CF800B904E0641C7B
:102B0000301EA6F10106F4D100BF2046F0BD30B55D
:102B100004460025204600F04AF870B1D4E90001CF
:102B2000401E814203D1A06838B1012505E0D4E9F7
:102B30000101401C814200D00125284630BD30B53E
:102B400004460025204600F032F820B1D4E90110F7
:102B5000884200D00125284630BD70B504460D4698
:102B600064B12068012809D90020A0602068401EB7
:102B700060602A462168E068FDF734FB70BD70B5DF
:102B800004460D46002685B12046FFF7C0FF60B120
:102B90006068401C60602168884201D3002060604A
:102BA0006168E068405C28700126304670BD0146CF
:102BB000002069B10A68012A0AD9CA6842B10B68C3
:102BC0008A689A4204D2D1E900329A4200D20120A6
:102BD000704770B504460D4600262046FFF7AFFF4C
:102BE00058B1A168481CA060E06845542168A068FD
:102BF000884201D30020A0600126304670BDF0B5A8
:102C00000A4600210023002400BF3DE0012505FA0B
:102C100001F3156805EA03049C4234D105684F00AE
:102C20000326BE40B543056015794E00B5400668E1
:102C3000354305601579012D02D01579022D16D185
:102C400085684F000326BE40B543856055794E0028
:102C5000B540866835438560456801268E40B5439A
:102C60004560456896798E40B6B235434560C56883
:102C70004F000326BE40B543C560D5794E00B54030
:102C8000C6683543C560491C1029BFD3F0BDF0B5F7
:102C9000002300244D07ED0E02FA05F3CE1000F1DB
:102CA000200555F826504E07F70E0F26BE40B543B7
:102CB000CF1000F1200646F82750CE1000F1200575
:102CC00055F8265045EA0304CE1000F1200545F8DA
:102CD0002640F0BD0246002013690B400BB10120D5
:102CE00000E0002070474183704701837047000077
:102CF0002DE9FC4105460C460027002600200090E7
:102D0000019055208DF80000422D01D1082000E0EF
:102D10000B208DF8010004208DF802008DF803408F
:102D200000208DF804008DF805009DF802109DF834
:102D3000032011449DF8042011449DF805208818B3
:102D4000C11700EB11610912A0EB0121C9B28DF886
:102D50000610BB208DF807003FE00821684601F00F
:102D600019F910211DA001F0D1F802F0E9FA00F5DF
:102D7000FA6720E01F48007801281CD100201D4977
:102D8000087012211CA001F0C1F8204800785528D5
:102D900011D11E4840780D280DD11C488078032899
:102DA00009D11A48C078A04205D1122118A001F01B
:102DB000ADF8BDE8FC81384602F0C8FA0028D9D148
:102DC000701CC6B2052E04DB102115A001F09EF880
:102DD000EFE7162118A001F099F8BEE753656E647D
:102DE0002047617261676520636F6E74726F6C0A51
:102DF00000000000F3040020476574205A69674210
:102E0000656520446174650A00000000E80900203F
:102E100047617261676520746F20580A00000000E6
:102E200047617261676520636F6E74726F6C2066B4
:102E300061696C65640A000072657472792E2E2EC9
:102E40000A00000010B50821074801F0A3F84FF46C
:102E5000967002F029FA0821044801F09BF86420DA
:102E600002F022FA10BD0000F60100200602002048
:102E700010B50446552027490870032048701020DB
:102E800088702078C87060780871A0784871897857
:102E9000204AD27811441F4A127911441D4A5279AE
:102EA0008818C11700EB11610912A0EB0121194A22
:102EB0009171BB201146C8710821104601F06AF8D3
:102EC0004FF4C87002F0F0F9112012498870E078D0
:102ED000C870207908716079487189780D4AD27874
:102EE00011440C4A127911440A4A52798818C117C0
:102EF00000EB11610912A0EB0121064A9171BB2080
:102F00001146C8710821104601F044F8642002F00F
:102F1000CBF910BDFF02002010B502210848FDF7D3
:102F20001DFB0748FDF71AFC00BF02210448FDF70E
:102F300085FB0028F9D00248FDF77CFB10BD00009E
:102F40000020014070B52DED068B012001F006F93F
:102F5000102001F003F900F097FB0F480478407847
:102F600000EB04242046FDF7C5F941EC1A0B9FED58
:102F70000B0B53EC102BFDF74EF941EC190BFDF741
:102F8000DDF908EE100ABDEEC80A10EE105AA8B21C
:102F9000BDEC068B70BD00005D0100203333333380
:102FA0003333F33F70B504460025002607E0FFF7F2
:102FB000B3FF0544052002F077F9701CC6B2A642A3
:102FC000F5DBB5FBF4F080B270BD000001460020D7
:102FD00021B107290AD008290ED10AE0074A527800
:102FE000064B1B7802EB032290B205E0034A5078AF
:102FF00002E0024A107800BF00BF7047980300202B
:1030000010B54FF480710248FFF764FE10BD000058
:103010000018024010B515480078012810D100F0C2
:10302000BFFE1349098888421EDB00200F49087043
:103030000320104908700021084600F075FF13E0D6
:103040000D48007801280FD100F0AAFE0849098830
:10305000884209DB002008490870032005490870F0
:103060000021084600F060FF10BD00005F03002053
:10307000780300206A0300206003002000B589B0B7
:103080000121212000F030FD09220B214248FFF7E9
:10309000FEFD09220C214048FFF7F9FD4FF4C05016
:1030A000079002208DF820008DF8210000208DF877
:1030B000220001208DF8230007A93748FFF79FFD64
:1030C0004FF48060079001208DF8200002208DF8D9
:1030D000210000208DF8220001208DF8230007A98F
:1030E0002E48FFF78CFD002000F05EF80121480615
:1030F00000F00AFD2A48FDF781FC00208DF816003B
:1031000001208DF8170000208DF8180001208DF89F
:10311000190000208DF81A0001208DF81B000020F6
:103120008DF812008DF8130001208DF81400022094
:103130008DF815000720ADF8100004A91848FDF718
:1031400006FD00208DF80A008DF80B0001208DF897
:103150000C000020ADF80000ADF80200ADF804004E
:10316000ADF80600ADF8080001208DF80D006846A6
:10317000FDF760FC12200B4908604860002048728F
:10318000087201208872002202210548FDF7D6FC52
:10319000FEF7AEFA09B000BD000002400014024084
:1031A00000640040F808002010B504462CB94FF424
:1031B00080610548FFF797FD04E04FF48061024805
:1031C000FFF793FD10BD00000014024010B5FEF79C
:1031D00039FE10BD10B504462CB14FF4807105487E
:1031E000FFF783FD04E04FF480710248FFF77BFD99
:1031F00010BD00000020024010B54FF4E06000F068
:103200009DFAA82002F032F801F038F900F028F811
:10321000FFF7F2FA01F015FFFFF730FFFDF7F2FAC2
:1032200000F01AFEFFF744FC01F024FD53210720B3
:10323000FEF7D8FDA72140F2E73002F09FF9A72161
:1032400040F2E73001F052F900F051FDFDF7D2FBFA
:1032500010BD0000014A10705170704798030020A3
:103260001CB50121202000F03FFC4FF400600090CD
:1032700001208DF8040000208DF8060001208DF853
:10328000070003208DF8050069460348FFF7B7FCE7
:103290000120024908601CBD00140240AC82424279
:1032A0002DE9F0410746884600202849086009209A
:1032B00001F0FAFF01202649C1F8AC02042001F018
:1032C000F3FF4FF40C7002F015F800242EE00025F7
:1032D00028E0385D284100F0010676B900201B493E
:1032E00008604FF4FA7002F005F801201849C1F89F
:1032F000AC024FF4FA7001F0FDFF012E10D1002056
:10330000124908604FF4FA7001F0F4FF01201049EF
:10331000C1F8AC0201F0C8FF4FF4487001F0EAFFB9
:10332000681CC5B2082DD4DB601CC4B24445CEDB9A
:103330000020064908604FF40C7001F0DBFF01200B
:103340000349C1F8AC02BDE8F0810000AC82424202
:103350000080424210B500F074FA08B1FE2010BDA2
:1033600000F05CFA022001F09FFF00F05DFA4120BE
:1033700000F054F908B1FE20F1E70120014908707E
:103380000020ECE78001002010B54A480068C0B971
:103390000A2001F089FF4748006890B94648006854
:1033A00008B9012000E000204349086000BF4148FF
:1033B00000680028FBD0F6204049087040A001F0CA
:1033C0002BFF3C48001D0068E0B90A2001F06CFFAB
:1033D0003848001D0068A8B93748001D006808B9C2
:1033E000012000E000203449091D086000BF314879
:1033F000001D00680028FAD0A6203049087034A0CB
:1034000001F00AFF2B4808300068B0B90A2001F02B
:103410004BFF28480830006878B927480830006812
:1034200008B9012000E0002023490831086000BFEE
:103430002048083000680028FAD01E480C30006888
:10344000B0BB0A2001F030FF1A480C30006878BB8E
:1034500019480C30006808B9012000E00020164926
:103460000C31086000BF13480C3000680028FAD007
:1034700040F6B8311420FFF747F94FF4967001F089
:1034800013FF5020FEF788FD4FF4967001F00CFFFB
:1034900040F6B8311420FFF737F94FF4967001F079
:1034A00003FF5020FEF778FD00210846FEF70CFDD3
:1034B00010BD000010024442B0824342420100208D
:1034C000BFAACABCB3C7CAD0D1B2BCEC00000000CE
:1034D000D6B4D0D0BCECB2E2C8CECEF10000000031
:1034E00010B5044655201F490870042048708870A4
:1034F0000020C870642094FBF0F00A2190FBF1F2E8
:1035000001FB1200174908710A2094FBF0F100FB3F
:10351000114194FBF0F00A2290FBF2F302FB13003E
:1035200001EB00100F49487189780E4AD278114496
:103530000C4A127911440B4A52798818C11700EBD2
:1035400011610912A0EB0121064A9171BB201146BD
:10355000C8710821104600F01DFD642001F0A4FE92
:1035600010BD0000FF020020F8B504460026002C24
:103570004BDD052C49DA642001F096FEFFF7E2FCF2
:10358000ADF80000002529E0701CC6B204212048D7
:10359000FFF786FE4FF4FA7001F086FE4FF4FA70E2
:1035A00001F082FE4FF4FA7001F07EFEFFF7CAFCD4
:1035B000ADF80200BDF80000BDF80210884207DA3D
:1035C000BDF80200ADF800000020ADF8020003E0F5
:1035D000C6F10500C6B203E0681CC5B2042DD3DBFA
:1035E00000BF022C04D104210948FFF759FE0CE06A
:1035F000032C04D104210748FFF752FE05E0042CF8
:1036000003D104210448FFF74BFE3046F8BD00000B
:10361000D2010020D6010020DA01002010B50446B6
:10362000412C25D108210846FFF722F93D21112020
:1036300001F09EFD8621172001F09AFD7F212620B2
:1036400001F096FD1E212D2001F092FD00212C207D
:1036500001F08EFD8D212A2001F08AFD3E212B20D4
:1036600001F086FD0A2001F01FFE00F0DDF801E008
:10367000FF2010BD0020FCE702468A4201D9501A03
:103680007047881AFCE7000010B5FDF77FF9472066
:10369000FDF750F900240EE0FDF702F9084908553E
:1036A000032C03D10120FDF725F902E00020FDF7EE
:1036B00021F9601CC4B2032CEEDBFDF783F910BDC9
:1036C0005D01002070B5002100230F22C4781CB3D7
:1036D000174C246804F4E064C4F5E064C4F30721E3
:1036E000C1F10404E3B20A4144789C40E1B2847819
:1036F000144021430C07210E0E4C057861550478C7
:1037000004F01F050124AC4005786D11AD0005F1F2
:10371000E025C5F8004109E0047804F01F05012404
:10372000AC40054D0678761145F8264070BD000086
:103730000CED00E000E400E080E100E0024901431C
:10374000024A1160704700000000FA050CED00E02D
:1037500000211148C079BB281CD10F4A92780E4B2A
:10376000DB781A440C4B1B791A440B4B5B79D0184D
:10377000C21700EB12621212A0EB0222D1B206486D
:103780008079884203D10120044A107002E00020B1
:10379000024A107070470000200900200605002032
:1037A00010B52DED048BB0EE080A164880ED000A26
:1037B00090ED000ADFED140A20EE200A80ED000AE9
:1037C0009FED120A124880ED000A90ED000ADFED2D
:1037D0000E0A20EE200A10EE101A0846FCF79BFD98
:1037E00041EC190B9FED0B0B53EC102BFCF713FD69
:1037F00041EC180BFCF7A2FD05490860BDEC048BF9
:1038000010BD0000BC0100200000C84200CC0D41EA
:10381000B8010020000000000070A74010B503218F
:103820001420FFF725F810BD10B5142000F04AFA57
:10383000044604F0030018B90321142000F0D0FB63
:1038400010BD10B500F01FFA08B1FE2010BD0F2109
:10385000012001F08DFC3D21112001F089FC1E2189
:103860002D2001F085FC00212C2001F081FC8D2110
:103870002A2001F07DFC3E212B2001F079FC402123
:10388000152001F075FC0020E0E7000010B50320D2
:10389000FFF788FB514908800846008800F06CFC5F
:1038A0004E4908804E4801884C480088FFF7E4FEE6
:1038B0004C4908704A480088F0BB4B48D0ED000ADC
:1038C0004648008800EE100AB8EE400A20EE800A52
:1038D000BCEEC00A10EE100A404908800846008875
:1038E00000EE100AB8EE400A4048D0ED000AB4EEEF
:1038F000E00AF1EE10FA03D200203D49087016E00C
:103900003648008800EE100AB8EE400A3748D0ED7D
:10391000000A30EE600ABCEEC00A10EE100A34490C
:10392000087008460078642801DD6420087030487B
:1039300000783049087000E004E008460178012072
:1039400000F0CEFA254800882549088025480078EF
:103950000A2842DD2448D0ED000A2048008800EE05
:10396000100AB8EE400A20EE800ABCEEC00A10EE43
:10397000100A1A4908800846008800EE100AB8EEBE
:10398000400A1A48D0ED000AB4EEE00AF1EE10FA4F
:1039900003D200201649087016E01048008800EE97
:1039A000100AB8EE400A1148D0ED000A30EE600A65
:1039B000BCEEC00A10EE100A0D49087008460078E7
:1039C000642801DD642008700948007809490870FE
:1039D00008460178012000F083FA10BDC2010020E2
:1039E000C4010020C6010020B8010020BC01002055
:1039F000C0010020B401002010B50446FF20144986
:103A0000087020204870207888706078C870A0788E
:103A10000871E078487106210D48FFF741FC4FF42A
:103A2000967001F041FC1020094948702079887097
:103A30006079C870A0790871E0794871062104485E
:103A4000FFF72EFC4FF4967001F02EFC10BD000025
:103A50001A03002010B586B004460121084600F084
:103A600043F80121102000F06FF8072209211B48BC
:103A7000FFF70DF907220A211848FFF708F94FF45C
:103A8000C060049002208DF8140000208DF816000C
:103A900001208DF8170003208DF8150004A90F48A8
:103AA000FFF7ADF800940020ADF80C000C20ADF845
:103AB0000A000020ADF80800ADF80600ADF80400DB
:103AC0006946074801F062F80121054800F0F6FF59
:103AD00000200449087006B010BD0000000002403C
:103AE000001001408001002029B1064A12680243FB
:103AF000044B1A6004E0034A12688243014B1A60C7
:103B0000704700003038024029B1064A126802436B
:103B1000044B1A6004E0034A12688243014B1A60A6
:103B2000704700004038024029B1064A126802433B
:103B3000044B1A6004E0034A12688243014B1A6086
:103B4000704700002038024029B1064A126802433B
:103B5000044B1A6004E0034A12688243014B1A6066
:103B6000704700004438024029B1064A12680243F7
:103B7000044B1A6004E0034A12688243014B1A6046
:103B80007047000024380240F0B5002100220024D4
:103B9000022500260223324F3F6807F00C0121B1B5
:103BA000042905D0082937D105E02E4F076036E0FB
:103BB0002D4F076033E02A4F3F1F3F68C7F3805601
:103BC000274F3F1F3F6807F03F036EB1264FB7FBFB
:103BD000F3F7DFF88CC0ACF1040CDCF800C0CCF3D8
:103BE000881C07FB0CF40CE01E4FB7FBF3F7DFF863
:103BF00070C0ACF1040CDCF800C0CCF3881C07FBEF
:103C00000CF4174F3F1F3F68C7F301477F1C7D002F
:103C1000B4FBF5F7076002E0124F076000BF00BF7A
:103C20000F4F3F6807F0F0010909104F7A5C0768F1
:103C3000D74047600A4F3F6807F4E051890A0B4FAD
:103C40007A5C4768D7408760054F3F6807F460415A
:103C5000490B064F7A5C4768D740C760F0BD00004B
:103C6000083802400024F40040787D014C03002015
:103C700001480078704700008001002010B5142032
:103C800000F020F810BD38B5FE250020009000247B
:103C900000BF12E0552000F089F942F21071684629
:103CA00000F032F838B9552000F080F9642001F0B6
:103CB000FBFA002503E0601C84B2642CEADB00BF41
:103CC00068B238BD38B5044604F03F0040F08004C7
:103CD000204600F06BF942F21071684600F014F8CB
:103CE00005460DB1FF2038BD9DF80000FBE710B57B
:103CF0004FF41650FFF7AEFE4FF4FA7001F0D4FA0D
:103D0000FFF728FB10BD000070B504460D4601F01A
:103D100017FB4FF4FA61B5FBF1F146180AE00A48C7
:103D2000008800F0200028B1074800F099FF2070BB
:103D3000002070BD304601F009FB0028EFD1034997
:103D400008700120F5E7000000100140800100200C
:103D500010B5FFF75FF901F05FFC01F03FFC00F0E8
:103D6000F5FB10BD00200749087007490870074996
:103D70000870074908700749087007490870074923
:103D8000087070475C0300205D0300205F03002083
:103D900060030020610300206A0300206303002009
:103DA0000F48B0F900000F4AB2F90020904207DD39
:103DB0000B48B0F900000B4AB2F90020811A06E066
:103DC0000848B0F90000064AB2F90020811AB1F59E
:103DD000004F02D94FF6FF70411A88B270470000B9
:103DE0009A030020800300200248B0F90000024935
:103DF000088070479A030020800300200248008852
:103E000002490880704700009C03002082030020C4
:103E10001CB58020009000208DF8040001208DF852
:103E2000070069460148FEF7EAFE1CBD0004024097
:103E30001CB58020009001208DF8040000208DF832
:103E4000060003208DF8050069460248FEF7D7FEFC
:103E50001CBD0000000402401CB54FF4E13000F02E
:103E6000C9FD01210220FFF73FFE4FF400700090D2
:103E700001208DF8040000208DF8060001208DF847
:103E8000070003208DF8050069460448FEF7B7FED9
:103E90004FF400710148FEF728FF1CBD00040240EA
:103EA00030B500228B071C0F0F2303FA04F20B4BD3
:103EB0008C1053F824309343084C8D1044F825306F
:103EC00023468C1053F824308C07240F00FA04F496
:103ED0002343024C8D1044F8253030BD0838014092
:103EE0007CB505460C4603208DF8040001208DF8B2
:103EF00005008DF8064000204FF4F073032201A95D
:103F000000901046FDF70AFB7CBD000070B504462A
:103F10000D462A4621460348FEF7E5FD642001F0E0
:103F2000C3F970BDEC0600207CB504460D46E0B236
:103F30008DF80400E0B28DF80500E8B28DF80600B7
:103F4000E8B28DF80700FDF7B7F978B10020034615
:103F500020220421009001A8FDF774F900202023FD
:103F6000024601A90090FDF7D9FA06E000202023BF
:103F7000042201A90090FDF7D1FA7CBD70B504467A
:103F80000D462A4621460248FEF7ADFD70BD0000F1
:103F90000C07002070B504460D462A46214602480B
:103FA000FEF7A1FD70BD00002C07002010B50446EF
:103FB0000A48008800BF0948008800F080000128F6
:103FC000F9D02146054800F050FE00BF40210348CB
:103FD00000F080FD0128F9D110BD00000010014063
:103FE00070B505460C4600262846FFF76BFE0646D0
:103FF00046EA0401284601F0BBF8002070BD00002D
:104000000CB50020019000903448006840F48030E6
:104010003249086000BF3148006800F40030009069
:104020000198401C0190009818B90198B0F5A04F74
:10403000F1D12A48006800F4003010B1012000904E
:1040400001E0002000900098012846D1234840302C
:10405000006840F0805021494031086020480068E5
:1040600040F440401E4908601C48083000681B4965
:10407000083108600846006840F4004008600846BF
:10408000006840F4A05008601648091F0860081F27
:10409000006840F08070091F086000BF0F4800688A
:1040A00000F000700028F9D040F205700E49086059
:1040B0000A480830006820F0030008490831086009
:1040C0000846006840F00200086000BF034808305E
:1040D000006800F00C000828F8D10CBD0038024040
:1040E0000070004019544007003C024010B50446DF
:1040F000012C04D141030548FEF7F5FD05E024B984
:104100004FF400510148FEF7F0FD10BD00080240D9
:1041100070B505460C46012D02D0022D1AD10CE0D7
:104120002CB14FF480610C48FEF7DDFD04E04FF444
:1041300080610948FEF7D9FD0CE02CB14FF4006115
:104140000548FEF7D0FD04E04FF400610248FEF799
:10415000CCFD00BF00BF70BD001C024010B504467E
:10416000FCF714FC4620FCF7E5FB2046FCF7E2FBDD
:10417000FCF728FC10BD000010B5024600230B48D8
:10418000828200210BE0094C481C34F8100024F80E
:104190001100204630F81100184483B2491C0A2946
:1041A000F1DB0A2093FBF0F080B210BD8406002002
:1041B000042808D14FF0E021096941F004014FF0D3
:1041C000E022116107E04FF0E021096921F00401CC
:1041D0004FF0E0221161704710B51548006840F4B7
:1041E0007000134908601348006840F0010011494D
:1041F000086000200F49083108600E4800680E4929
:1042000008400C4908600D48091D0860081F006837
:1042100020F48020091F0860002006490C31086046
:10422000FFF7EEFE4FF0006001498039086010BDD5
:1042300088ED00E000380240FFFFF6FE1030002459
:1042400070B505460C46552022490870422D02D112
:104250000820487002E00B201E49487050201D497C
:1042600088700020C870642094FBF0F00A2190FB55
:10427000F1F201FB1200174908710A2094FBF0F1DA
:1042800000FB114194FBF0F00A2290FBF2F302FBD9
:10429000130001EB00100F49487189780D4AD2785C
:1042A00011440C4A127911440A4A52798818C117EC
:1042B00000EB11610912A0EB0121064A9171BB20AC
:1042C0001146C87108211046FFF764FE642000F013
:1042D000EBFF70BDFF02002010B50121054800F082
:1042E00056F8012801D1FFF733FD0121014800F004
:1042F0003FF810BD0040014010B50121074800F013
:1043000046F8012804D106480068401C04490860AA
:104310000121024800F02CF810BD000000440140CB
:104320004403002010B50121074800F030F80128AF
:1043300004D106480068401C044908600121024875
:1043400000F016F810BD000000100040CC01002065
:1043500010B50121054800F01AF8012801D1FEF737
:1043600035FF0121014800F003F810BD00140040A2
:10437000CA430282704721B1028842F001020280E2
:1043800004E002884FF6FE731A400280704730B591
:104390000246002000230024158A05EA01039589BE
:1043A00005EA010413B10CB1012000E0002030BD8A
:1043B0001AB183890B43838102E083898B43838114
:1043C0007047000000220288184B98420ED0184B0C
:1043D00098420BD0B0F1804F08D0164B984205D0D0
:1043E000154B984202D0154B984204D14FF68F736B
:1043F0001A404B881A43124B984207D0114B9842EF
:1044000004D04FF6FF431A400B891A4302804B68D1
:10441000C3620B880385054B984202D0044B984237
:1044200001D18B7A0386012383827047000001400B
:10443000000401400004004000080040000C00405F
:1044400000100040001400401CB501210420FFF7BB
:104450004BFB4FF40050009001208DF804008DF8C4
:10446000070069460448FEF7CAFB4FF400510248B2
:10447000FEF73BFC1CBD00000008024010B500F038
:1044800005F8FFF7E1FF00F017F810BD1CB501219A
:104490004020FFF729FB4FF48070009000208DF83A
:1044A000040001208DF8070069460248FEF7A7FBCB
:1044B0001CBD0000000002401CB501218020FFF758
:1044C00013FB4FF44060009001208DF804008DF83C
:1044D000070069460448FEF792FB4FF4406102482A
:1044E000FEF703FC1CBD0000001C02407FB5054622
:1044F0000C4601214804FFF727FB0295ADF8044064
:104500000020ADF80600ADF80C008DF80E0001A9F2
:104510000D48FFF757FF19208DF8000000208DF897
:10452000010006208DF8020001208DF80300684686
:10453000FFF7C8F8012211460348FFF739FF0121B0
:104540000148FFF718FF7FBD0044014010B5064841
:104550000078012806D10820FEF738FDC4B22046B5
:1045600000F004F810BD00006103002010B50446FF
:1045700054B900207A49087001207A490870002156
:104580000846FFF7D1FC86E0E72C08D176480068A2
:104590007649086074480068754908607BE0F72C2C
:1045A00001D0F32C0AD17048006814306F490860BC
:1045B0006D48006828386E4908606CE0FB2C01D01B
:1045C000F92C0AD1684800682830684908606648B4
:1045D00000683C38664908605DE0FD2C01D0FC2C89
:1045E0000AD1614800683C30604908605E48006854
:1045F0005A385F4908604EE0FE2C0AD15A480068DC
:1046000050305A490860584800687838584908605E
:1046100041E0EF2C01D0CF2C0AD153480068143070
:10462000534908605048006828385049086032E013
:10463000DF2C01D09F2C0AD14B48006828304C4910
:104640000860494800683C384849086023E0BF2CAE
:1046500001D03F2C0AD1444800683C3044490860EE
:10466000414800685A384149086014E07F2C0AD15B
:104670003D48006850303E4908603B480068783843
:104680003A49086007E03848006838490860364809
:104690000068374908603748007801282FD17E2C00
:1046A0000BD03E2C09D07C2C07D0C32C05D0782C05
:1046B00003D040F61E6084420BD1002028490870C8
:1046C0000120284908702C49087000210846FFF78E
:1046D0002BFC04F01800182811D104F0800010B150
:1046E00004F0010058B900201D49087001201D493F
:1046F00008702149087000210846FFF715FCFF2CBF
:1047000020D11948006819490860174800681849FD
:1047100008601A480088B0F5966F0DDD0020174933
:10472000088000210846FFF7FFFB00200C490870B5
:1047300004200C49087008E010480088401C0F490C
:10474000088002E000200D4908800548007828B163
:104750000748016805480068FEF799F810BD000099
:10476000610300206A030020740300206C03002012
:10477000700300206403002063030020680300200E
:10478000024600215178107840EA0121084670471E
:10479000024600211178507840EA0121084670470E
:1047A00010B5024800F0A6FB10BD0000F405002083
:1047B00010B51248007800BB40F22551104800F0B7
:1047C00096F9012819D10E4800F04AFA0D490E4A0F
:1047D000127888540C480078401C0B490870084631
:1047E0000078022804DB00200870012003490870CB
:1047F00040F22551024800F052F910BD5901002045
:10480000001001405B0100205A01002010B540F269
:104810002551184800F06BF901282AD11648007874
:1048200090B900F08DFD0A30144908600020144949
:104830000870104800F014FA1249114A127888548E
:1048400001200D4908700FE00D480078C8280BDAE8
:10485000084800F005FAC1B209480078401CC0B20F
:10486000074A1070074A115440F22551014800F0E0
:1048700016F910BD00440040F1040020F8040020A7
:10488000F00400202009002000B587B00121042099
:10489000FFF72AF901212020FFF756F90822062107
:1048A0002348FEF7F4F9082207212148FEF7EFF923
:1048B000C020059002208DF8180000208DF81A0005
:1048C00003208DF8190001208DF81B0005A9184858
:1048D000FEF795F94FF4E13001900020ADF810009B
:1048E0000C20ADF80E000020ADF80C00ADF80A0069
:1048F000ADF8080001A90F4800F048F9012240F284
:1049000025510C4800F01DF947208DF800000020CB
:104910008DF801008DF8020001208DF80300684633
:10492000FEF7D0FE0121034800F0C8F807B000BD33
:10493000000802400014014010B540F225512848FB
:1049400000F0D5F8002845D0254800F089F9254920
:1049500008702548007878B908460078552839D17C
:104960000120214908701F48007820490870002064
:1049700048708870C8702DE01B480078012807D166
:10498000022019490870174800781849487021E03A
:1049900015480078022807D10320134908701148F0
:1049A00000781249887015E00F48007803280AD172
:1049B00000200D4908700B4800780C49C870012090
:1049C0000B49087006E00020074908700849087084
:1049D0000649087040F22551014800F060F810BD0A
:1049E00000140140200300202103002022030020A6
:1049F0002A03002010B586B0044601210420FFF7E9
:104A000073F801212020FFF79FF8082206211D4896
:104A1000FEF73DF9082207211A48FEF738F9C020B1
:104A2000049002208DF8140000208DF8160001205B
:104A30008DF8170003208DF8150004A91148FEF722
:104A4000DEF800940020ADF80C000C20ADF80A0050
:104A50000020ADF80800ADF80600ADF80400694686
:104A6000094800F093F80121074800F027F8402199
:104A7000054800F00BF82021034800F007F806B0C5
:104A800010BD0000000802400014014001F4007253
:104A9000B2F5007F00D100BFCA430280704710B555
:104AA0000022002340F66A14A14200D100BF0A127E
:104AB00001249440A3B2DC43048010BD21B182895B
:104AC00042F40052828104E082894DF6FF731A405D
:104AD0008281704702460020B1F5007F00D100BFFF
:104AE00013880B400BB1012000E00020704770B527
:104AF0000246002400230025002040F66A16B14239
:104B000000D100BFC1F3421501F01F03012606FAD0
:104B100003F3012D02D19689334006E0022D02D124
:104B2000168A334001E0968A33400C12012606FAB9
:104B300004F41688344013B10CB1012000E00020C9
:104B400070BDF0B50346002400260025002040F685
:104B50006A17B94200D100BF1846C1F3421401F0F0
:104B60001F06012707FA06F5012C01D10C3004E0DD
:104B7000022C01D1103000E014301AB107682F4325
:104B8000076002E00768AF430760F0BD2DE9FF470B
:104B900005460E460024A14600BFA046B08900B1DC
:104BA00000BF2C8A24F44054F08804432C82AC8942
:104BB00041F20C608443B08831890843718908430D
:104BC0000443AC81AC8A24F44074B0890443AC82C1
:104BD0006846FEF7D9FF2048854202D01F4885422B
:104BE00002D1DDF80C9001E0DDF80890A88900F40E
:104BF000004040B109EBC90000EB091031684900E1
:104C0000B0FBF1F707E009EBC90000EB09103168D0
:104C10008900B0FBF1F76420B7FBF0F00401200934
:104C2000642101FB1078A88900F4004040B13220D3
:104C300000EBC800B0FBF1F000F00700044308E00F
:104C4000322000EB08106421B0FBF1F000F00F00FF
:104C500004432C81BDE8FF8700100140001401408F
:104C600001468888C0F308007047C1F308028280BB
:104C70007047000010B512481249C1F8B000322147
:104C80001048C0F8B4100021C0F8B810C0F8BC102B
:104C9000C0F8C0100C49C0F8C4100221C0F8C810F8
:104CA0000021C0F8CC10C0F8D010C0F8D4100421F6
:104CB00080F8D81000200549087000F081F810BD78
:104CC0001005002044050020620100206101002041
:104CD00070B505460C46E1B2044A284600F01EF8BD
:104CE00014B101200249087070BD0000F4050020D5
:104CF0006101002010B5034800F02EF800200249A1
:104D0000087010BDF40500206101002010B50248B4
:104D100000F03EF810BD0000F405002070B5034619
:104D2000002013E0D2E90154AC4206D21D5C966823
:104D3000741C94601468A55506E0064D1469AC42D5
:104D400002D21469641C1461441CE0B28842E9DB9D
:104D500070BD0000F0FFFF7F10B5044694F82810E6
:104D60000A4A52F82100002240F22771FFF7E9FEBB
:104D70000020A060E060206194F82810034A52F8F7
:104D8000210040F22771FFF78AFE10BD6801002064
:104D900010B504460020E0602068007894F82810E0
:104DA000064A52F82110888094F8281052F8210001
:104DB000012240F22771FFF7C4FE10BD68010020F8
:104DC00000B587B0012140F20910FEF78DFE0121E8
:104DD0004FF42020FEF798FE082200214048FDF7FE
:104DE00056FF072206213F48FDF751FF00208DF8AE
:104DF0001A0001208DF81B0002208DF818000120F8
:104E0000059002208DF8190005A93548FDF7F7FE39
:104E100002208DF818004020059005A93148FDF7C3
:104E2000EEFE00208DF81A0001208DF81B008DF891
:104E300018000002059002208DF8190005A92A48E3
:104E4000FDF7DDFE0020FEF7C5F94FF4E1300190DB
:104E50000020ADF80800ADF80A00ADF80C00ADF880
:104E600010000820ADF80E0001A92048FFF78EFEC3
:104E700001211E48FFF722FE34208DF8000000209B
:104E80008DF8010002208DF8020001208DF803004A
:104E90006846FEF717FC4FF4E13001900420ADF8AE
:104EA0000E0001A91248FFF771FE26208DF80000C0
:104EB00000208DF801008DF8020001208DF803001C
:104EC0006846FEF7FFFB012240F225510848FFF734
:104ED00038FE01210648FFF7F1FD07B000BD0000D4
:104EE00000000240000C024000200240004C004044
:104EF0000044004010B5044694F82810374A52F890
:104F0000210040F22771FFF7F2FD18B3E068401C62
:104F1000E060D4E90210884209D2E1682068405C70
:104F200094F828102D4A52F82110888009E094F84E
:104F300028102A4A52F82100002240F22771FFF778
:104F400000FE94F82810254A52F8210040F22771FB
:104F5000FFF7A5FD94F82810204A52F8210040F2EE
:104F60002551FFF7C4FD30B300F0EAF9606294F810
:104F700028001A4951F8200080881949087094F8CF
:104F80002810164A52F8210040F22551FFF787FDFC
:104F9000D4E90610884207D211480178E269501C12
:104FA000E0616069815406E00E49206A884202D2BD
:104FB000206A401C206294F82810084A52F8210008
:104FC0000821FFF787FD38B194F82800034951F80C
:104FD000200080880449087010BD0000680100208E
:104FE00064010020F0FFFF7F650100200EB54FF443
:104FF000C060FEF7A3FB01218803FEF7A5FD042195
:105000000120FEF74DFF1020019000208DF80800D0
:105010000C208DF8090001208DF80A0001A8FDF789
:10502000FDFC0A208DF8000000208DF8010007200B
:105030008DF8020001208DF803006846FEF742FB60
:105040000EBD10B500F008F85321092000F064F8F7
:10505000FFF7CCFF10BD00001CB501210320FEF7B7
:1050600043FD00220E211448FDF711FE00220D2100
:105070001148FDF70CFE4FF40040009001208DF820
:10508000040000208DF8060001208DF807000320A1
:105090008DF8050069460848FDF7B1FD1020009025
:1050A00000208DF8040001208DF8070069460348B0
:1050B000FDF7A5FD1CBD00000000024000040240F9
:1050C00010B5012010490860032000F013F90020FA
:1050D0000E49C1F8BC0201210D48FFF74CF901212E
:1050E0000B48FFF745F900200A4908601E2000F030
:1050F000DBF8012004490860052000F0D5F8002104
:105100000348FFF738F910BDBC024042000040429E
:1051100000100040CC0100207FB505460C4601215F
:105120001020FEF7F1FC0295ADF804400020ADF828
:10513000060001A90D48FFF745F936208DF800005B
:1051400000208DF8010008208DF8020001208DF864
:1051500003006846FEF7B6FA012211460348FFF73E
:1051600027F900210148FFF706F97FBD0010004034
:1051700070B504460D462946204600F001F870BD82
:10518000F8B504460D46032704F03F04002714E059
:105190002046FEF70BFF42F210716846FEF7B4FDA1
:1051A000064646B99DF80000844203D12846FEF722
:1051B000FDFE04E00226781CC7B2032FE8DB00BF27
:1051C0003046F8BD70B504460D46552011490870AB
:1051D0000620487008468470C57000200871487128
:1051E00089780C4AD27811440A4A12791144094A42
:1051F00052798818C11700EB11610912A0EB012147
:10520000044A9171BB201146C87108211046FEF76F
:10521000C1FE70BD3003002070B505462846FAF780
:10522000F3FF84B2A01C000A07494870A01C8870D4
:1052300005210548FEF7AEFEE1B22846FEF7AAFEBC
:10524000642000F031F870BD2B03002002E008C894
:10525000121F08C1002AFAD170477047002001E0F0
:1052600001C1121F002AFBD17047000010B504468F
:105270006FF00400FEF79CFFE11704EB5171C1F3DE
:10528000C701074A11701046007800EB4001C1EBDE
:10529000C0104FF6FF7101EAC0000249088010BD3E
:1052A0003E030020400300200146114A12884A4371
:1052B0004FF0E0235A6100229A611A46126942F0C7
:1052C00001021A6100BF4FF0E022106900F00102F4
:1052D0001AB100F48032002AF5D04FF0E0221269B2
:1052E00022F001024FF0E0231A6100229A61704718
:1052F000400300200146114A12784A434FF0E02350
:105300005A6100229A611A46126942F001021A613A
:1053100000BF4FF0E022106900F001021AB100F462
:105320008032002AF5D04FF0E022126922F001020B
:105330004FF0E0231A6100229A6170473E0300207B
:1053400001480068704700004403002004490968D0
:10535000884203D902490968401A00E000207047DA
:105360004403002000240025FDF746FFFFF7E8FF77
:10537000323074490860FFF7E3FFC83072490860B3
:10538000FFF7DEFFC83071490860FFF7D9FFC8306A
:105390006F49086055206F490870AA204870552051
:1053A0006D4908700220487000210846FEF7BCFDD8
:1053B000C6E0FDF7E9FFFCF7B1F9FCF7DFFBFCF70E
:1053C0001FFE60480068FFF7C1FF60B9FFF7B8FF34
:1053D00032305C4908606148006808B9012000E08B
:1053E00000205E49086058480068FFF7AFFF30B9F9
:1053F000FFF7A6FFC83054490860FEF747FA544843
:105400000068FFF7A3FF20BBFFF79AFFC8305049A1
:105410000860FEF72DFC60B9FEF769FC4F4828389C
:10542000006808B9012000E000204C4928390860D4
:105430000FE000204949283908604948D0F8B002F7
:1054400008B9012000E0002044490C390860FEF74B
:1054500015FC3E480068FFF779FF002870D1FFF780
:105460006FFF00F5FA70394908603E48007800285F
:105470004FD13D48007837498870FDF7C1FD354967
:10548000C870FFF71DFE39490888C11700EB11618C
:105490000912A0EB01212F4A117134490888C11764
:1054A00000EB1161090A5171FDF74CFD04462046DD
:1054B000E11704EB11610912A4EB0121254A917156
:1054C000E11704EB1161090AD1712948008885B2FE
:1054D0002846E91705EB11610912A5EB01211172AC
:1054E000E91705EB1161090A51722248007811464B
:1054F00088720D211046FEF741FDFFF7FBFB0D21E1
:105500001448FFF7E5FBFFF701FC0020194908707C
:1055100016E014480078012812D1174800780128B5
:105520000ED1FFF7E7FB32210B48FFF7D1FBFFF766
:10553000EDFB32210848FEF721FD00200E490870DE
:1055400037E70000300100202C010020340100204A
:10555000380100202006002052060020BC82434271
:1055600000804342F40400206A030020D0010020A0
:105570009A03002045010020F50400207FB5054670
:105580000C4601210804FEF7DFFA0295ADF804404D
:105590000020ADF80600ADF80C008DF80E0001A952
:1055A0000D48FEF70FFF18208DF8000000208DF841
:1055B000010005208DF8020001208DF803006846E7
:1055C000FEF780F8012211460348FEF7F1FE0121A3
:1055D0000148FEF7D0FE7FBD0040014010B5002419
:1055E0000A48007880B1FEF7DBFB044608480088D3
:1055F000844209DB00200549087002200549087033
:1056000000210846FEF790FC10BD00005E0300205C
:105610007A0300206A03002010B500242648007891
:10562000012822D10820FDF7D1FC04460320FFF712
:105630003BFE04F0100080B92048006832283AD9B7
:1056400000201D4908701D49086002201C4908708F
:1056500000210846FEF768FC2DE0FF2C2BD11748EF
:105660000068401C1549086025E0164800780128AC
:1056700021D10820FDF7AAFC04460320FFF714FE01
:1056800004F0080080B90D480068322813D90020C2
:105690000C49087009490860022009490870002176
:1056A0000846FEF741FC06E0FF2C04D103480068E1
:1056B000401C0249086010BD5C0300207C030020F0
:1056C0006A0300205D0300200100000002000000CA
:1056D000040000000800000010000000200000008E
:1056E00040000000800000000001000000020000F7
:1056F000000400000008000000100000002000006E
:1057000000400000008000000000010000000200D6
:10571000000004000000080000001000000020004D
:1057200000004000000080000000000100000002B6
:10573000000000040000000800000010000000202D
:105740000000004000000080FEFFFFFFFDFFFFFFA4
:10575000FBFFFFFFF7FFFFFFEFFFFFFFDFFFFFFF95
:10576000BFFFFFFF7FFFFFFFFFFEFFFFFFFDFFFF0C
:10577000FFFBFFFFFFF7FFFFFFEFFFFFFFDFFFFF75
:10578000FFBFFFFFFF7FFFFFFFFFFEFFFFFFFEFFEB
:10579000FFFFFBFFFFFFF7FFFFFFEFFFFFFFDFFF55
:1057A000FFFFBFFFFFFF7FFFFFFFFFFEFFFFFFFDCC
:1057B000FFFFFFFBFFFFFFF7FFFFFFEFFFFFFFDF35
:1057C000FFFFFFBFFFFFFF7F0008040C020A060E69
:1057D0000109050D030B070FF85700080000002012
:1057E00010050000FE0400084459000810050020C0
:1057F000A00900005C520008102200FF0CF300FF1B
:1058000018E700FF5EA103051445DE92673478A215
:10581000FD27FF1401000000FF14020610045503C9
:10582000010D1302BB08110F1203084220081304D4
:1058300003182204085200101118200505BB550E4C
:105840003C1201083302011830040E020228300411
:105850000E020320520F20520F20520F20520F2011
:10586000520D70520D7030040D01034040040D01C3
:1058700004205158520D585205305205305205300F
:10588000520530520530520588130B10B82211080A
:1058900011B0500512BB550A70521018200702A013
:1058A000A1000041081005A200004208D008A5A2EE
:1058B000A000E7BB000100062A28321801000110F1
:1058C0000A10014000440040004804124C041250E9
:1058D0000C414B9012303132333435363738394140
:1058E0004243444546FF01000E21524649445F4170
:1058F0004444523A30310A6605FFD20528D2062ABE
:1059000008BE16FD0275F012FA010611A1E320058A
:10591000010203040400063F060708090001100AFB
:10592000C003E0078002E007A0041007E000E007E2
:105930000001081104A12406FF30F20D3AC403E16E
:045940000100000062
:040000050800018965
:00000001FF
